:103C9E000ECF0EBB0EA70E920E7C0E650E4D0E3481
:103CAE000E190DFE0DE10DC40DA50D850D640D4211
:103CBE000D1E0CFA0CD40CAE0C860C5D0C330C08DD
:103CCE000BDC0BB00B820B540B250AF50AC40A93BE
:103CDE000A610A2F09FD09CA09960963092F08FC12
:103CEE0008C808950861082E07FB07C807960764E1
:103CFE000733070206D206A206730645061705EA23
:103D0E0005BF059305690540051704F004C904A312
:103D1E00047E045A0437041503F403D303B4039644
:103D2E000378035B033F0324030A02F002D702BFAA
:103D3E0002A80292027C02670253023F022C021A70
:103D4E00020801F701E601D601C701B801A9019CDD
:103D5E00018E018101740168015D01510146013C32
:103D6E0001320128011F0115010D010400FC00F4B0
:103D7E0000EC00E500DE00D700D000CA00C300BD95
:103D8E0000B800B200AD00A700A2009E00990094FA
:103D9E000090008C008700840080007C0078007505
:103DAE000072006E006B0068006500620060005DCE
:103DBE00005A0058005500530051004E004C004A66
:103DCE0000480046004400430041003F003E003CD6
:103DDE00003A00390037003600350033003200312A
:103DEE00002F002E002D002C002B002A0029002869
:103DFE000027002600250024002300010C010104E9
:103E0E0002011E030A96040132050303060064072D
:103E1E00010108000009015A0E01010F00011200F4
:103E2E006413010114013C1501FA1664FA17FFFF21
:103E3E001D00072000072400022701012F013C303E
:103E4E00010132010335FFFF3603073CFFFF3DFF43
:103E5E00FF180002191E461A00021B00022D32C85E
:103E6E002E0001FAFAFA18000019FFFF1A00001BC3
:0B3E7E0000002D32C82E0001FAFAFAF5
:10004800900786E0FEA3E0FF7457BE0010D39F40E0
:100058000C903E0812001EE493F599802F9000142E
:10006800E0D394044014900786E0FEA3E0FF903E9E
:100078000812001EE493F5998012900786E0FEA30B
:10008800E0FF903E1D12001EE493F599900786123A
:10009800000E900786E0FEA3E0FF746C6F4E7003BD
:1000A80075130022900072E0B40208740190007287
:1000B800F0D20D90013AE090002AF090013BE090D8
:1000C800002BF090013CE090002CF0A20AB34016FF
:1000D80090013AE0700C90013BE0700690013CE022
:1000E80060028002C20A90013AE0B4300F90013BEE
:1000F800E0B4470890013CE0643B60028004D20C05
:100108008002C20CE558B40102800302022E90005E
:1001180057E0F566900062E0F568900063E0F569E5
:10012800900074E0F56A90007AE0900029F0900061
:100138007CE0F56590007DE0F567900080E0F5646F
:10014800900081E0F563900090E0900041F090000D
:1001580091E0900042F0900092E0900043F090000F
:1001680093E0900044F0900094E0900045F09000F7
:1001780095E0900046F0900096E0900047F09000DF
:1001880097E0900048F0900099E0900033F09000DC
:100198009AE0900034F090009BE0900035F09000D9
:1001A8009CE0900036F0900079E0B4011790000AC6
:1001B800740FF0A374FFF090000CE4F0A3F0740245
:1001C800900079F0900079E0B4035990000CE0FEBB
:1001D800A3E0FF90000AE0FCA3E0FD120003741006
:1001E800123FE97408123FDBEF900026F0EF70062B
:1001F80074FF900026F07400900079F090000BE0F6
:10020800900027F090000AE0900028F0900026E087
:10021800900789F0900027E090078AF0900028E086
:1002280090078BF0803F900081E07006755801754B
:100238006300A20AB3402E90013AE090002AF090A1
:10024800013BE090002BF090013CE090002CF090F6
:10025800002AE0700C90002BE0700690002CE06003
:10026800028002C20AE5667003756602E5687003DB
:100278007568027E887F4DE5668E048F05FF123F04
:10028800CB8C398D3AE56975F0FAA4FFAEF0E568D4
:100298008E048F05FF123FCB8C3D8D3E90004FE0C2
:1002A800F56090004DE0FE900069E0B506189000FA
:1002B8004CE0FE900068E0B5060C90004BE0FE9024
:1002C8000059E06E606F900069E07006900068E089
:1002D80060067400900059F0900069E0B40208903C
:1002E80000497401F08005900049E4F0900068E04E
:1002F800B4020890004A7401F0800590004AE4F0C6
:10030800900068E0600690004AE060028005756031
:10031800038003756004E559B55802D20D90006852
:10032800E090004CF0900069E090004DF09000598A
:10033800E090004BF0740190009EF0740190009FD3
:10034800F074009000A0F074009000A1F074009088
:1003580000A2F074009000A3F074009000A4F07460
:10036800019000A5F074019000A6F074009000A719
:10037800F074009000A8F074009000A9F074009048
:1003880000AAF074009000ABF074019000ACF07417
:10039800019000ADF074009000AEF074009000AFD2
:1003A800F074009000B0F074009000B1F074009008
:1003B80000B2F07401900362F07401900363F0746A
:1003C80000900364F07400900365F0740090036675
:1003D800F07400900367F07400900368F074009064
:1003E80003A2F074019003A3F074019003A4F074C5
:1003F800009003A5F074009003A6F074009003A782
:10040800F074009003A8F074009003E2F074009078
:1004180003E3F074019003E4F074009003E5F074D2
:10042800009003E6F074009003E7F074009003E88E
:10043800F07401900422F07400900423F074019089
:100448000424F07400900425F07400900426F074DD
:1004580000900427F07400900428F022E5B554F7C2
:10046800F5B5E5B554FDF5B5C2A2C2A1C292C20761
:10047800C297C2A0E5B554FBF5B5755104E5510422
:10048800F55290004FE0F560900025E4F0C209E5D0
:10049800B554FEF5B522750A00750900AE09AF0A14
:1004A8007457BE00039F500302055B903E0812007C
:1004B8001EE49390004E1240010FBF00010EE0FCB5
:1004C800903E0812001EECFEE493FFEEC39F5026F8
:1004D800AE09AF0A0FBF00010E903E0812001EAE13
:1004E80009AF0AE493FC903E0812001EE4939000C2
:1004F8004E124001ECF0AE09AF0A903E0812001E01
:10050800E49390004E124001E0FC903E0A12001E57
:10051800ECFCE493FDECD39D4019903E0A12001EBA
:10052800E493FC903E0812001EE49390004E1240A3
:1005380001ECF0AE09AF0A74022FFF50010E8E09CC
:100548008F0A780A740126F6500418E436F6400338
:100558000204A422750A00750900AE09AF0A7415D1
:10056800BE00039F5003020629903E5F12001EE45E
:100578009390004E1240010FBF00010EE0FC903E28
:100588005F12001EECFEE493FFEEC39F5026AE09F7
:10059800AF0A0FBF00010E903E5F12001EAE09AFFA
:1005A8000AE493FC903E5F12001EE49390004E1202
:1005B8004001ECF0AE09AF0A903E5F12001EE493D2
:1005C80090004E124001E0FC903E6112001EECFCCF
:1005D800E493FDECD39D4019903E6112001EE49314
:1005E800FC903E5F12001EE49390004E124001EC16
:1005F800F0AE09AF0A740F6F4E7006750A157509CB
:1006080000AE09AF0A74022FFF50010E8E098F0A3F
:10061800780A740126F6500418E436F640030205F9
:100628006222750A00750900AE09AF0A7415BE008A
:10063800039F50030206F7903E7412001EE4939045
:10064800004E1240010FBF00010EE0FC903E7412F4
:10065800001EECFEE493FFEEC39F5026AE09AF0ADE
:100668000FBF00010E903E7412001EAE09AF0AE4DF
:1006780093FC903E7412001EE49390004E124001C9
:10068800ECF0AE09AF0A903E7412001EE49390009D
:100698004E124001E0FC903E7612001EECFCE49302
:1006A800FDECD39D4019903E7612001EE493FC9019
:1006B8003E7412001EE49390004E124001ECF0AE1E
:1006C80009AF0A740F6F4E7006750A15750900AEEA
:1006D80009AF0A74022FFF50010E8E098F0A780A9B
:1006E800740126F6500418E436F640030206302258
:1006F800054D22054C22054EC2CF2290F800E49306
:100708006406600280FE75840175A70075FF8090FD
:100718000788E4F075C91075A70F75A1C775A700FC
:1007280075D90075CEFF75A70F75F1FE75F2FF75C7
:10073800F33775F47875A4BA75A5FF75A60775AE75
:100748000075AFFF75D48175D5FF75D6FF75D7FFD6
:10075800C296C295C2A0C20BC297E5B554BFF5B503
:10076800E5B554DFF5B5E5B554EFF5B5E5B5547F16
:10077800F5B5E5B554F7F5B5E5B554FDF5B575A787
:100788000075A20175A14775F80975BC0175BE040D
:1007980075BD6C75BE0775BDA075BE0875BD0175C4
:1007A800BC0075BB1875BC2075BA0875E88075D192
:1007B8001375A70F75E10575E20075C740759700B9
:1007C800759780740A123FBB7597C0E597542070DF
:1007D8000280F8758F0275A700D2AF75980075A9C9
:1007E8000C75A70F75AB4375ADFB75AC1E75A700EF
:1007F800758911758E00758C00758A00D2A9D28C06
:10080800758D00758B00D2ABD28E75CD0075CC007E
:1008180075CA0075CB00D2ADC2CFD2CA7591047526
:1008280092007593CD75EF0675D94075CF01900785
:1008380086E4F0A3F0751300751400C299D20A7407
:10084800C8F5187517001225C775A70FE5FB9000A6
:100858001AF0E5FA90001BF0E5F990001CF075A776
:100868000090F800E493F5081226FE122C38900741
:1008780089E0900026F090078AE0900027F0900722
:100888008BE0900028F090078CE0900029F090070A
:100898008DE0F56690078EE0F56890078FE0F569C2
:1008A800900790E0F56A900791E0F565900792E06F
:1008B800F567900793E0F564900794E0F563900777
:1008C80095E090002AF0900796E090002BF09007B2
:1008D80097E090002CF0900798E0900041F0900786
:1008E80099E0900042F090079AE0900043F090075A
:1008F8009BE0900044F090079CE0900045F0900742
:100908009DE0900046F090079EE0900047F0900729
:100918009FE0900048F09007A0E0900033F0900727
:10092800A1E0900034F09007A2E0900035F0900725
:10093800A3E0900036F07400900082F090013AE055
:10094800700C90013BE0700690013CE0600280046E
:10095800C20A8002D20A90F807E493900021F0902E
:100968000021E0440A900021F0900021E054FE901C
:100978000021F07406900012F07402900013F090B9
:10098800F802E493900014F07403900015F07403D7
:10099800900016F07406900017F07405900018F097
:1009A800900014E0B404067404900018F0740490E5
:1009B8000019F090F804E49390001DF07400900082
:1009C8001EF090F805E49390001FF090F806E49369
:1009D800900020F074FF900022F07447900125F0F9
:1009E800744D900126F07420900127F07434900122
:1009F80028F0744C900129F0743690012AF0743074
:100A080090012BF0744590012CF0742090012DF08A
:100A1800742090012EF0742090012FF0743490010E
:100A280030F07453900131F07450900132F07444F6
:100A3800900133F090007AE0D3940140067400905E
:100A4800007AF0755801755901740390004CF01242
:100A580000AC12049E900014E0B4040512062A802B
:100A68000312055C1225F3E5B554FEF5B590002593
:100A7800E4F0900786E4F0A3F07524007523007570
:100A88004800752A007529007549007532007531CE
:100A980000754A00755400755500755A0075510463
:100AA80075520175343C753300757000756F0075AB
:100AB80071CD7572CD755600755700754300754434
:100AC80000754500754600755B0075470075420066
:100AD800754100900006E4F0A3F0900008E4F0A34C
:100AE800F0755E00755F0090000E74FDF0A374E869
:100AF800F0900023E4F07464900024F0C200D20166
:100B0800C202D203754D00756D00C294C293C287AC
:100B1800C290C291C20D7E017F00900028E0123F72
:100B2800E9900027E02FFF50010E90000AEEF0A395
:100B3800EFF0900026E0700674FF900026F0900019
:100B48000AE0FEA3E0FFEFD394FFEE940F40079076
:100B5800000AE4F0A3F07400900071F074009000B3
:100B680079F07400900082F0740090008DF07400A9
:100B78009000B4F0E5677003756704743A90074E07
:100B8800F074FD90074FF09003D4E0900414F0D275
:100B9800B0D2B7D2A7D2A6D2B1D2A3C207A2B6B357
:100BA8009204A2B3B39205D29CD2EC75CF01A2985D
:100BB800B34005C298122F9CE5136006A299B3B3FF
:100BC80040028005C299123512E51464016005E5FA
:100BD80014B4040280D5E54DD39405400CE55AC3FE
:100BE80094C85002055A754D00E571C394FA501A1D
:100BF800786F12003FAE6FAF70EFD394E8EE9403B6
:100C080040080571757000756F00C28E7E047F0004
:100C1800E54C123FE9E58D75F004A4FDACF0EF2D2D
:100C2800FDEE3CFCE58B75F04084FF7E00ED2FFF68
:100C3800EC3EFE8E258F26D28EA2B6300401B3502C
:100C480003020D79A2B6300401B35003020D79A254
:100C5800B6405A0554E5B54401F5B5900024E4F0D2
:100C6800E554D3956640447C887D4D123E898E2399
:100C78008F24E5482FFF50010E7401123FDB8E23AD
:100C88008F24852448755401C28E758D00758B009C
:100C9800754C00D28E7403BE00039F500690002549
:100CA8007401F0E543B40603754300D204A2B6B359
:100CB8005003020D79C20490006BE060181236539D
:100CC800A200B34008E5B54408F5B58006E5B5547B
:100CD800F7F5B58002C20090006EE060181237A8E0
:100CE800A202B34008E5B54402F5B58006E5B5545F
:100CF800FDF5B58006E5B554FDF5B5A207B340048A
:100D0800D2878002C287900059E06004D2908002A6
:100D1800C29090004AE0B40104D2948002C2949038
:100D28000049E0B40104D2938002C293A209B340FF
:100D380004D2918002C291900018E0FE900014E065
:100D4800C39E4009900014E0D39408400974FB90B6
:100D58000023F012046490001DE0601590001DE06F
:100D6800FE900017E06E600974FE900023F01204F4
:100D780064C2CA7E017F00E54E123FE9E5CD2FFF30
:100D880050010E8E278F28D2CAE565B4014890001D
:100D98000EE0FCA3E0FDEFC39DEE9C4039B208E5F0
:100DA8002A45296013A208B34008E5B54404F5B5FF
:100DB8008006E5B554FBF5B590000EE0FEA3E0FF14
:100DC800900010E0FCA3E0FDEF2DFDEE3CFC900050
:100DD8000EECF0A3EDF0A2B3300501B35003020E00
:100DE800BEA2B3300501B35003020EBEA2B3500336
:100DF800020EB70555E5B54401F5B5900024E4F0B9
:100E0800E555D395685003020EB57CEA7D60AE27A0
:100E1800AF28123E898E298F2AE569123FE974FFAF
:100E28008E048F05FF123FCB8C298D2AE5492DFDB5
:100E380050010C74018C068D07123FDB8E298F2A16
:100E4800852A49A209B340157464123FE9900067E6
:100E5800E08E048F05FF123FCB8C298D2A75550132
:100E680090000EE0FEA3E0FFAC27AD28120003902F
:100E7800000EEEF0A3EFF0E567FF123FCB740AFF18
:100E8800123FCB90007BE08C068D07123FE974146B
:100E98008E048F05FF123FCB900010ECF0A3EDF00D
:100EA800C2CA75CD0075CC00754E00D2CAD205A253
:100EB800B3B34002C205900025E0B40107E556C36C
:100EC800940640030214CFE56D9025A6F8282873F0
:100ED800900059E0C39402400302102CE551D394CA
:100EE80001500302102CE55175F040A4FFAEF090BC
:100EF800031212001EE0C395455018E55175F040E5
:100F0800A4FFAEF090031112001EE0F52E752D001F
:100F180002102CE55175F040A4FFAEF090031012BA
:100F2800001EE0C395454003020FC8E55175F04027
:100F3800A4FFAEF090031112001EE55175F040A415
:100F4800FFAEF0E0FC90030F12001EECFEE0FFEE97
:100F5800C39FFEE5518E0475F040A4FFAEF09003E8
:100F68001012001EE0F40425458C0088F0A4FFAEA2
:100F7800F0E5518F048E0575F040A4FFAEF09003A4
:100F88001212001EE55175F040A4FFAEF0E0FA9091
:100F9800031012001EEAFEE0FFEEC39FFECDCCCD8B
:100FA8008E07123FCBE55175F040A4FFAEF09003D9
:100FB8000F12001EE02DFD50010C8C2D8D2E80642B
:100FC800E55175F040A4FFAEF090030F12001EE546
:100FD8005175F040A4FFAEF0E0FC90030E12001E25
:100FE800ECFEE0FFEEC39F8545F0A4FFAEF0E551AF
:100FF8008F048E0575F040A4FFAEF0900310120028
:101008001EE0FECDCCCD8E07123FCBE55175F040EA
:10101800A4FFAEF090030E12001EE02DFD50010C4F
:101028008C2D8D2E756D010214CF900059E0C3945C
:101038000240030211DF90004FE0D39551500302A4
:101048001188E55175F040A4FFAEF0900318120026
:101058001EE0C395455018E55175F040A4FFAEF069
:1010680090031712001EE0F52C752B00021188E57D
:101078005175F040A4FFAEF090031612001EE0C3B5
:1010880095454003021124E55175F040A4FFAEF0E8
:1010980090031712001EE55175F040A4FFAEF0E072
:1010A800FC90031512001EECFEE0FFEEC39FFEE568
:1010B800518E0475F040A4FFAEF090031612001E86
:1010C800E0F40425458C0088F0A4FFAEF0E5518FCC
:1010D800048E0575F040A4FFAEF090031812001EB0
:1010E800E55175F040A4FFAEF0E0FA900316120047
:1010F8001EEAFEE0FFEEC39FFECDCCCD8E07123F69
:10110800CBE55175F040A4FFAEF090031512001E18
:10111800E02DFD50010C8C2B8D2C8064E55175F071
:1011280040A4FFAEF090031512001EE55175F04083
:10113800A4FFAEF0E0FC90031412001EECFEE0FFEA
:10114800EEC39F8545F0A4FFAEF0E5518F048E05F0
:1011580075F040A4FFAEF090031612001EE0FECD1D
:10116800CCCD8E07123FCBE55175F040A4FFAEF011
:1011780090031412001EE02DFD50010C8C2B8D2CB9
:10118800E551B40122E560D39401401BE551C395B4
:10119800565014E545C39405500D90035FE0A82907
:1011A800B80006952A40028003755102E551B560E2
:1011B8002290004FE0D395514019E55175F040A4B5
:1011C800FFAEF090031712001EE0A823B8000695A2
:1011D80024400280020560756D020214CF90005908
:1011E800E0B4022AE55175F040A4FFAEF090031771
:1011F80012001EE0F52C752B00E55175F040A4FF98
:10120800AEF090030E12001EE0F52E752D00900032
:1012180059E0B4030F900051E0F52C752B00752EA2
:1012280000752D00756D030214CFE55175F040A4CB
:10123800FFAEF090032012001EE0C3955A4003024F
:101248001306900049E07036E551D394014029AE69
:1012580023AF24AC2DAD2EEDD39FEC9E401AE55163
:1012680075F040A4FFAEF090031E12001EE0A829FE
:10127800B80005D3952A5002800215518034E551F3
:10128800D394024029AE23AF24AC2DAD2EEDD39FCD
:10129800EC9E401AE55175F040A4FFAEF090031E95
:1012A80012001EE0A829B80005D3952A5002800232
:1012B8001551E551B55236E551C39560502FE551AA
:1012C800C395565028AE23AF24AC2BAD2CEFD39D3D
:1012D800EE9C4019E55175F040A4FFAEF090031F55
:1012E80012001EE0A829B80006952A4002800205CF
:1012F80051C292E55165526005C207755A00756D75
:10130800040214CFE55175F040A4FFAEF090031A23
:1013180012001EE0B40117E55175F040A4FFAEF0CD
:1013280090032012001EE0240AC3955A40030213BA
:10133800DC753064752F00A207B3500B900060E095
:101348002405C3954540030213DCE55175F040A41C
:10135800FFAEF090031D12001EE0C395454064E502
:101368005175F040A4FFAEF090031C12001EE55129
:1013780075F040A4FFAEF0E0FC90031B12001EECD9
:10138800FEE0FFEEC39F8545F0A4FFAEF0E5518F68
:10139800048E0575F040A4FFAEF090031D12001EE8
:1013A800E0FECDCCCD8E07123FCBE55175F040A4C1
:1013B800FFAEF090031B12001EE02DFD50010C8CB7
:1013C8002F8D30AE23AF24AC2FAD30EFD39DEE9CE4
:1013D8004002D207756D050214CFE551B40109909A
:1013E8000059E0C3940240030214AF900358E0D3BD
:1013F800954550030214AF900356E0C395455040FD
:10140800900357E0FE900355E0F4042EFE90035637
:10141800E0F40425458E0088F0A4FFAEF090035850
:10142800E0FC900356E0F4042C8E048F05FF123F75
:10143800CB900355E02DFD50010C8C2B8D2C802C6E
:10144800900355E0FE900354E0F4042E8545F0A483
:10145800FFAEF0900356E08E048F05FF123FCB904D
:101468000354E02DFD50010C8C2B8D2CE551C395B8
:1014780060502FE551C395565028AE23AF24AC2BAE
:10148800AD2CEFD39DEE9C4019E55175F040A4FFBB
:10149800AEF090031F12001EE0A829B80006952A96
:1014A80040028003755102900049E0B40106E551FD
:1014B800640160028003755102E55165526005C2FE
:0714C80007755A00756D0065
:1025A600020ED80210320211E502123202130C0298
:0225B60013E22E
:1014CF00900050E02402A823B80007D395244002CF
:1014DF00C207900025E0B40109900059E0C39403BE
:1014EF004003021655900049E060030215A5E5512F
:1014FF00D394014034E55175F040A4FFAEF0900352
:10150F001412001EE0A823B8001FD39524401AE53B
:10151F005175F040A4FFAEF090031F12001EE0A81B
:10152F0029B80005D3952A500280021551E551D3F1
:10153F009401402FE55175F040A4FFAEF0900312D7
:10154F0012001EE0C39545501AE55175F040A4FFF7
:10155F00AEF090031E12001EE0A829B80005D39527
:10156F002A500280021551E551D394014021E551D3
:10157F00D39556401AE55175F040A4FFAEF0900395
:10158F001E12001EE0A829B80005D3952A5002802C
:10159F0002155102164AE551D394024034E55175B4
:1015AF00F040A4FFAEF090031412001EE0A823B881
:1015BF00001FD39524401AE55175F040A4FFAEF0FB
:1015CF0090031F12001EE0A829B80005D3952A50DA
:1015DF000280021551E551D39402402FE55175F069
:1015EF0040A4FFAEF090031212001EE0C3954550C9
:1015FF001AE55175F040A4FFAEF090031E12001EC5
:10160F00E0A829B80005D3952A500280021551E5AC
:10161F0051D394024021E551D39556401AE55175A7
:10162F00F040A4FFAEF090031E12001EE0A829B8F0
:10163F000005D3952A500280021551E5516552607D
:10164F0005C207755A00900060E0D3954550099088
:10165F000054E0C395455002C207900059E0700353
:10166F000218B8A2A5B34008A2A4B340030218A160
:10167F00AE35AF367441D39F749C9E4005783512BA
:10168F00003FAE35AF36EFB48806EEB413028003D9
:10169F0002187EA2A55003021741900059E0B40131
:1016AF000B90004FE0D3956040020560900059E029
:1016BF00B40253E55175F040A4FFAEF09003201231
:1016CF00001EE0C3955A503E90004FE0D395514015
:1016DF0020E551C395565019E55175F040A4FFAE62
:1016EF00F090031412001EE0A823B80006952440C2
:1016FF00028002055190004FE0F560E551655260A0
:10170F0005C207755A00900059E0B4032590004FA9
:10171F00E0D395514007E551C3955640028002052D
:10172F005190004FE0F560E55165526005C20775B5
:10173F005A00A2A4500302187E900059E0B4016E23
:10174F00900049E07035E551D394014029E551757A
:10175F00F040A4FFAEF090031E12001EE0A829B8BF
:10176F00000FD3952A400A1551755A008551608094
:10177F000385516080037560018033E551D3940276
:10178F004029E55175F040A4FFAEF090031E120002
:10179F001EE0A829B8000FD3952A400A1551755A93
:1017AF000085516080038551608003756002900051
:1017BF0059E0D394015003021872E55175F040A41B
:1017CF00FFAEF090032012001EE0C3955A400302B3
:1017DF001872900049E07041E551D394014034E50F
:1017EF005175F040A4FFAEF090031112001EE0A857
:1017FF0023B8001FD39524401AE55175F040A4FF7C
:10180F00AEF090031E12001EE0A829B80005D39574
:10181F002A500280021551803FE551D39402403483
:10182F00E55175F040A4FFAEF090031112001EE0D9
:10183F00A823B8001FD39524401AE55175F040A492
:10184F00FFAEF090031E12001EE0A829B80005D3CA
:10185F00952A500280021551E55165526005C20765
:10186F00755A00E556B40704055E8003755E00E502
:10187F0063B4010EAE35AF36EF64407005EE649C75
:10188F006002800EA2A54003755801A2A440037503
:10189F005802A2A5B3B35006A2A4B3B34002800668
:1018AF007536007535000219A6A2A5B34008A2A48B
:1018BF00B34003021992AE35AF367441D39F749C77
:1018CF009E4005783512003FAE35AF36EFB488062F
:1018DF00EEB413028003021992A2A5406F90006824
:1018EF00E0605A90004AE0B4010790004AE4F080AB
:1018FF000690004A7401F090004AE070057560038D
:10190F00800375600490004AE0B40104D294800211
:10191F00C294E551B4041AE55175F040A4FFAEF03E
:10192F0090031E12001EE0A829B80005D3952A5077
:10193F00028008755103C207755A00800375600451
:10194F00E556B40704055E8003755E00A2A440331C
:10195F00900069E06021900049E0B40107900049D0
:10196F00E4F080069000497401F0900049E0B40162
:10197F0004D2938002C293E556B40704055E800338
:10198F00755E00A2A5B3B35006A2A4B3B340028004
:10199F0006753600753500E558655960069000826A
:1019AF00E06003021B2EC29C751400751300C2CA9F
:1019BF00E5589025B8F82828738012122C38800D1E
:0D19CF00122D118008122DEA8003122EC384
:0F25B8000219C80219CA0219CF0219D40219D97F
:1019DC00900029E090007AF0E566900057F0E568F9
:1019EC00900062F0E569900063F0E56A900074F095
:1019FC00E56590007CF0E56790007DF0E564900073
:101A0C0080F0E563900081F090002AE090013AF0BC
:101A1C0090002BE090013BF090002CE090013CF00A
:101A2C00900041E0900090F0900042E0900091F026
:101A3C00900043E0900092F0900044E0900093F00E
:101A4C00900045E0900094F0900046E0900095F0F6
:101A5C00900047E0900096F0900048E0900097F0DE
:101A6C00900033E0900099F0900034E090009AF0F0
:101A7C00900035E090009BF0900036E090009CF0D8
:101A8C007400900082F07447900125F0744D900121
:101A9C0026F07420900127F07434900128F0744CD7
:101AAC00900129F0743690012AF0743090012BF0DB
:101ABC00744590012CF0742090012DF0742090014D
:101ACC002EF0742090012FF07434900130F0745388
:101ADC00900131F07450900132F07444900133F065
:101AEC009003D4E0900414F0743A90074EF074FD17
:101AFC0090074FF01200AC900004E4F0A3F09000BB
:101B0C00067475F0A37430F09000087475F0A3742B
:101B1C0030F0855859D2CA754C00D29C741B900079
:101B2C0023F0E556C394065005E551B55202806783
:101B3C00C207E55175F040A4FFAEF09003221200ED
:101B4C001EE030E003D38001C39296E55175F0405E
:101B5C00A4FFAEF090032312001EE030E003D3800C
:101B6C0001C39295E55175F040A4FFAEF0900324AB
:101B7C0012001EE030E003D38001C3920B8551525A
:101B8C00AE29AF2A7405BE00039F5007E545D394D8
:101B9C000550028002D292E556D394055003021CE4
:101BAC00ADC207E551D394014073E55175F040A4E3
:101BBC00FFAEF090031E12001EE0A829B80007D358
:101BCC00952A40021551E5516552604EE55175F06C
:101BDC0040A4FFAEF090032212001EE030E003D3CD
:101BEC008001C39296E55175F040A4FFAEF09003CE
:101BFC002312001EE030E003D38001C39295E5511F
:101C0C0075F040A4FFAEF090032412001EE030E00B
:101C1C0003D38001C3920B855152021CADE556B41F
:101C2C0006279000ACE030E003D38001C39296907D
:101C3C0000ADE030E003D38001C392959000AEE09C
:101C4C0030E003D38001C3920BE556B40727900014
:101C5C00A5E030E003D38001C392969000A6E0305B
:101C6C00E003D38001C392959000A7E030E003D34A
:101C7C008001C3920BE556B4082790009EE030E03B
:101C8C0003D38001C3929690009FE030E003D38091
:101C9C0001C392959000A0E030E003D38001C39281
:101CAC000B900072E06058E54575F00284FF7E00F1
:101CBC0090014E12001EE0F55CE54775F00A84FFBA
:101CCC007E0090024E12001EE0F55DE55C255DD3B2
:101CDC009464400BE55C255DC39464F55C800375EE
:101CEC005C00E55C75F00284FF7E008F5CEFC394B2
:101CFC00335007EF24CDF55C8003755CFF801CE549
:101D0C004575F00284FF7E0090014E12001EE075B6
:101D1C00F00284FF7E00EF24CDF55CE55CD394EB00
:101D2C004003755CEBE595C3955C4004C2A2800250
:101D3C00D2A2E556D394054002C207A2074007750C
:101D4C0071CDC2978002D297E595C395714004C2BC
:101D5C00A18002D2A1A20BB340057572FA80037563
:101D6C0072CDE595C395724004C2A08002D2A0E565
:101D7C0043C39406400302237EA2EDB35003022317
:101D8C007EC2EDE5436003021EE07E017F00E5BEEE
:101D9C00123FE9E5BD2FFF50010E900000EEF0A3BD
:101DAC00EFF0900029E0B401177E0F7FFF90000048
:101DBC00E0FCA3E0FD120003900000EEF0A3EFF0B6
:101DCC00900079E0B4025B900000E0FEA3E0FF908D
:101DDC00000AE0FCA3E0FDEDD39FEC9E400F9000C9
:101DEC0000E0F8A3E090000AC8F0A3C8F09000004F
:101DFC00E0FEA3E0FF90000CE0FCA3E0FDEFD39D20
:101E0C00EE9C400F900000E0F8A3E090000CC8F0AE
:101E1C00A3C8F0900000E0FEA3E0FF7404123FDBC7
:101E2C008F44900079E07060900000E0FEA3E0FF2A
:101E3C0090000AE0FCA3E0FDEFD39DEE9C400D1258
:101E4C000003900000EEF0A3EFF08007900000E498
:101E5C00F0A3F0900000E0FEA3E0FF7410123FE945
:101E6C00900026E08E048F05FF123FCB900000EC13
:101E7C00F0A3EDF07400D39D74019C400890000118
:101E8C00E0F54480037544FFE54475F00AA4FFAE09
:101E9C00F074198E048F05FF123FCB8D45ED253262
:101EAC00FFAE3150010E7401123FDB8F4585453278
:101EBC00753100EFD394624003754562900072E077
:101ECC0064016006900066E0600280057543018045
:101EDC000375BB17E543B401028003021FD07E01DA
:101EEC007F00E5BE123FE9E5BD2FFF50010E9000CB
:101EFC0000EEF0A3EFF0900072E0B4017EE5344503
:101F0C00336025AC33AD341DBDFF011C8F028E0335
:101F1C008C068D07903C9E12002EE493FE74019368
:101F2C00FFEFC39AEE9B400280057833124013AE4C
:101F3C0033AF3474B3BE0025D39F4021900000E032
:101F4C00FCA3E0FD0FBF00010E903C9E12002EE49E
:101F5C0093FE740193FFEDC39FEC9E4002800578C5
:101F6C003312003FAE33AF34E56A123FE974648E2E
:101F7C00048F05FF123FCB8D478033900066E060E5
:101F8C002D900000E0FEA3E0FFEFD39400EE940848
:101F9C00400F900066E0B40104C2098002D20980AF
:101FAC000D900066E0B40104D2098002C2099000D1
:101FBC0072E064026006900066E0600575BB1680F6
:101FCC0003754302E543B4020280030220BE7E0186
:101FDC007F00E5BE123FE9E5BD2FFF50010E9000DA
:101FEC0000EEF0A3EFF0900072E0B4027EE5344511
:101FFC00336025AC33AD341DBDFF011C8F028E0345
:10200C008C068D07903B3412002EE493FE740193E2
:10201C00FFEFC39AEE9B400280057833124013AE5B
:10202C0033AF3474B3BE0025D39F4021900000E041
:10203C00FCA3E0FD0FBF00010E903B3412002EE418
:10204C0093FE740193FFEDC39FEC9E4002800578D4
:10205C003312003FAE33AF34E56A123FE974648E3D
:10206C00048F05FF123FCB8D478033900066E060F4
:10207C002D900000E0FEA3E0FFEFD39400EE940857
:10208C00400F900066E0B40104C2098002D20980BE
:10209C000D900066E0B40104D2098002C2099000E0
:1020AC0072E07003754700900066E07002C209751B
:1020BC00BB1FE543B403457E017F00E5BE123FE93B
:1020CC00E5BD2FFF50010E900000EEF0A3EFF07471
:1020DC0009123FE974E68E048F05FF123FCB8C4149
:1020EC008D42E54A2DFD50010C74018C068D0712B2
:1020FC003FDB8E418F4285424A75BB19E543B404E0
:10210C000280030222667E017F00E5BE123FE9E5F4
:10211C00BD2FFF50010E900000EEF0A3EFF0740401
:10212C00123FDB8F4BE564B4010280030221F3758F
:10213C006B00756B00E56BD3940740030221E0E55F
:10214C006B900041124001E0D3954B501AE56B9017
:10215C000041124001E0F404254BFEE56B90003782
:10216C00124001EEF08017E56B900041124001E047
:10217C00C3954BFEE56B900037124001EEF0E56B1A
:10218C00C394044009900084E0C3956B503BE56B0D
:10219C006029E56B900037124001FEE0FFEE9000E5
:1021AC003FE0D39F4013E56B900037124001E09065
:1021BC00003FF0E56B900040F0800E900037E0900F
:1021CC00003FF07400900040F0786B740126F640EC
:1021DC0003022141900040E0F4042408F556E55632
:1021EC00D394054002C292E564D39401402FE54B91
:1021FC00D3946E4004D20E8002C20E755605E5646F
:10220C00B40205A20EB340028003755607E564B410
:10221C000306A20EB3B340028003755607E557655B
:10222C00566008E55104F552855657E556B4070833
:10223C00E5B54480F5B58006E5B5547FF5B5E556B2
:10224C0064066005E556B40808E5B54410F5B5809C
:10225C0006E5B554EFF5B575BB13E543B40502803F
:10226C000302237A7E017F00E5BE123FE9E5BD2F14
:10227C00FF50010E900000EEF0A3EFF07404123F3B
:10228C00DB8F46E563B402028003022377756B0093
:10229C00756B00E56BD39403400302232EE56B9022
:1022AC000033124001E0D39546501AE56B90003391
:1022BC00124001E0F4042546FEE56B90002D12401F
:1022CC0001EEF08017E56B900033124001E0C395EE
:1022DC0046FEE56B90002D124001EEF0E56B602997
:1022EC00E56B90002D124001FEE0FFEE900031E016
:1022FC00D39F4013E56B90002D124001E09000310C
:10230C00F0E56B900032F0800E90002DE0900031E3
:10231C00F07400900032F0786B740126F6400302E2
:10232C00229F900082E07043E52A45296036E558EB
:10233C00C39403500A900032E004C394034002801B
:10234C0007900032E004F558E558D39402400A9007
:10235C000032E004D3940250028007900032E00473
:10236C00F5588007900032E004F55875BB1805430A
:10237C00D2ECE55ED39404500302247F75CF01C2E6
:10238C00A2AE35AF367488D39F74139E4005A2A5B8
:10239C00B34014AE35AF367488D39F74139E40058A
:1023AC00A2A4B340028048783512003FAE35AF3658
:1023BC00EFB4883BEEB41337A2A5B3500990004F8D
:1023CC00E0D395515002800405518011A2A5B35061
:1023DC000890004FE0655160028002D207A2A4B3BE
:1023EC005007E551D39401500280041551C207A245
:1023FC00A5B3B35006A2A4B3B34002800675360051
:10240C00753500E5516552604EE55175F040A4FFFD
:10241C00AEF090032212001EE030E003D38001C323
:10242C009296E55175F040A4FFAEF0900323120094
:10243C001EE030E003D38001C39295E55175F04066
:10244C00A4FFAEF090032412001EE030E003D38012
:10245C0001C3920B855152A20740057571CD8003C3
:10246C007571FFE595C395714004C2A18002D2A19C
:10247C00022388AE25AF26EFD39420EE944E500362
:10248C0002257A120464C28E758D00758B00754C12
:10249C0000D28EC207757000756F007571CD7551C5
:1024AC0004752400752300755400755A00C287907A
:1024BC000059E06004D2908002C29090004AE0B4CF
:1024CC000104D2948002C294900049E0B40104D279
:1024DC00938002C293A209B34004D2918002C291AC
:1024EC0090006BE06018123653A200B34008E5B5BB
:1024FC004408F5B58006E5B554F7F5B58002C20081
:10250C0090006EE060181237A8A202B34008E5B53F
:10251C004402F5B58006E5B554FDF5B58006E5B584
:10252C0054FDF5B590000E74FDF0A374E8F0E5438E
:10253C00B40603754300900025E4F075260075255C
:10254C0000758D00758B00754C00900024E0C394D1
:10255C00035008900024E004F080067403900024DB
:10256C00F0900024E0B40306E5B554FEF5B5AE27B3
:10257C00AF28EFD39410EE9427401CC2CA75CD003F
:10258C0075CC00752800752700D2CA754E00752AC7
:0A259C0000752900755500020BB30D
:10395A000000010001320164019601960200021280
:10396A0002240200020003000340038003C0040093
:10397A000440048004C00500060006000600060094
:10398A00060006000600060000FF013101630195EA
:10399A0001FF01FF0211022302FF02FF02FF033FA0
:1039AA00037F03BF03FF043F047F04BF04FF05FF37
:1039BA0006FF06FF06FF06FF06FF06FF06FF06FFD5
:1039CA000FAA0FA50F9F0F9A0F940F8D0F870F80C5
:1039DA000F780F710F680F600F570F4E0F450F3B8F
:1039EA000F300F250F1A0F0E0F020EF50EE80EDB21
:1039FA000ECC0EBE0EAE0E9F0E8E0E7D0E6C0E5AA5
:103A0A000E470E340E200E0C0DF70DE20DCB0DB540
:103A1A000D9D0D850D6D0D540D3A0D200D050CE90A
:103A2A000CCE0CB10C940C760C580C3A0C1B0BFBFC
:103A3A000BDB0BBB0B9A0B790B570B350B130AF1EC
:103A4A000ACE0AAB0A870A640A400A1C09F809D492
:103A5A0009B0098C09670943091F08FB08D608B28F
:103A6A00088E086A0846082307FF07DC07B9079685
:103A7A0007730751072F070D06EC06CA06AA06891F
:103A8A0006690649062A060A05EC05CD05B005921F
:103A9A0005750558053C0520050504EA04CF04B55B
:103AAA00049C04820469045104390422040B03F4BB
:103ABA0003DE03C803B2039D038903750361034D43
:103ACA00033B03280316030402F202E102D102C0F7
:103ADA0002B002A0029102820273026502570249F1
:103AEA00023C022F02220216020901FD01F201E63E
:103AFA0001DB01D001C601BB01B101A7019D0194FF
:103B0A00018B01820179017001680160015801503D
:103B1A000148014101390132012B0125011E011819
:103B2A000111010B010500FF00FA0FA60FA00F9962
:103B3A000F920F8B0F840F7C0F740F6B0F620F584D
:103B4A000F4E0F430F380F2C0F1F0F120F050EF7D2
:103B5A000EE80ED80EC80EB70EA50E930E800E6C88
:103B6A000E580E420E2C0E150DFD0DE40DCB0DB1A7
:103B7A000D950D790D5D0D3F0D200D010CE10CC069
:103B8A000C9E0C7C0C590C350C100BEA0BC40B9ECA
:103B9A000B760B4F0B260AFD0AD40AAA0A800A558D
:103BAA000A2A09FF09D409A8097C0950092508F934
:103BBA0008CD08A10875084A081E07F307C8079D1B
:103BCA0007730749072006F706CE06A6067E06579C
:103BDA000630060A05E405BF059B0577055405323C
:103BEA00051004EF04CE04AE048F047104530435A7
:103BFA00041903FD03E203C703AD0394037B0363C4
:103C0A00034B0334031E030802F302DE02CA02B6A0
:103C1A0002A30291027F026D025C024C023C022C5A
:103C2A00021D020E020001F201E401D701CA01BE1F
:103C3A0001B101A6019A018F0185017A017001661D
:103C4A00015D0153014A0141013901310129012173
:103C5A0001190112010B010400FD00F700F000EA4E
:103C6A0000E400DE00D900D300CE00C900C400BFC2
:103C7A0000BA00B500B100AD00A800A400A0009CE5
:103C8A00009900950091008E008A008700840081C7
:043C9A00007E007B2D
:1025C700751A00751900AE19AF1AAC17AD18EDC31F
:1025D7009FEC9E401674FF123FBB75CF01781A74AB
:1025E7000126F6500418E436F650DB22900786E4FD
:1025F700F0A3F0751000750F00751300751400C275
:102607000FD21022C2AF75D900758F0375B7A575A4
:10261700B7F190F800E4F0758F0175B7A575B7F1BC
:10262700E50890F800F075B7A575B7F190F801E4E3
:10263700F075B7A575B7F190079DE090F802F075B2
:10264700B7A575B7F19007A1E090F803F075B7A5A6
:1026570075B7F190079EE090F804F075B7A575B7C8
:10266700F190079FE090F805F075B7A575B7F19061
:1026770007A0E090F806F075B7A575B7F19007A227
:10268700E090F807F0758F0075D940D2AF22900718
:1026970088E0B4AB61C2AF75D90075B62275F52273
:1026A700758F0375B7A575B7F1740090F600F075CF
:1026B7008F01750A00750900AE09AF0A7413BE00D1
:1026C700279F402475B7A575B7F190078912001E9B
:1026D700E0FC90F60012001EECF0780A740126F672
:1026E700500418E436F650D0758F0075F51175B69D
:1026F7002075D940D2AF22C2AF75D90075F52275C2
:102707000A00750900AE09AF0A7413BE00229F4084
:102717001F90F60012001EE493FC90078912001E1A
:10272700ECF0780A740126F6500418E436F650D512
:1027370075F51175D940D2AF22900788E0B4AA0287
:10274700800302287DC2AF75D90075B62275F522C0
:10275700758F0375B7A575B7F1740090EE00F07526
:10276700B7A575B7F1740090F000F075B7A575B708
:10277700F1740090F200F075B7A575B7F174009089
:10278700F400F0758F01750A00750900AE09AF0AEC
:1027970074FFC39F74019E402475B7A575B7F19068
:1027A700004E12001EE0FC90EE0012001EECF078C6
:1027B7000A740126F6500418E436F650CF750A005D
:1027C700750900AE09AF0A74FFC39F74019E4024C8
:1027D70075B7A575B7F190024E12001EE0FC90F098
:1027E7000012001EECF0780A740126F6500418E473
:1027F70036F650CF750A00750900AE09AF0A74FFA7
:10280700C39F74019E402475B7A575B7F190044E18
:1028170012001EE0FC90F20012001EECF0780A7421
:102827000126F6500418E436F650CF750A007509EC
:1028370000AE09AF0A74FFC39F74019E402475B7A9
:10284700A575B7F190064E12001EE0FC90F4001239
:10285700001EECF0780A740126F6500418E436F6E8
:1028670050CF758F0075F51175B62075D940D2AF69
:10287700743A90074EF022900788E0B4AA028003CA
:102887000229BBC2AF75D90075B62275F522758FBF
:102897000375B7A575B7F1740090E600F075B7A595
:1028A70075B7F1740090E800F075B7A575B7F174C6
:1028B7000090EA00F075B7A575B7F1740090EC00C9
:1028C700F0758F01750A00750900AE09AF0A74FF2C
:1028D700C39F74019E402475B7A575B7F190004E4C
:1028E70012001EE0FC90E60012001EECF0780A745D
:1028F7000126F6500418E436F650CF750A0075091C
:1029070000AE09AF0A74FFC39F74019E402475B7D8
:10291700A575B7F190024E12001EE0FC90E8001278
:10292700001EECF0780A740126F6500418E436F617
:1029370050CF750A00750900AE09AF0A74FFC39F2F
:1029470074019E402475B7A575B7F190044E120027
:102957001EE0FC90EA0012001EECF0780A740126D3
:10296700F6500418E436F650CF750A00750900AE24
:1029770009AF0A74FFC39F74019E402475B7A575FC
:10298700B7F190064E12001EE0FC90EC0012001EFC
:10299700ECF0780A740126F6500418E436F650CFA6
:1029A700758F0075F51175B62075D940D2AF743A99
:1029B70090074EF022900788E0B4AA028003022A0B
:1029C700F9C2AF75D90075B62275F522758F0375F3
:1029D700B7A575B7F1740090DE00F075B7A575B7A8
:1029E700F1740090E000F075B7A575B7F174009029
:1029F700E200F075B7A575B7F1740090E400F075C3
:102A07008F01750A00750900AE09AF0A74FFC39FED
:102A170074019E402475B7A575B7F190004E12005A
:102A27001EE0FC90DE0012001EECF0780A7401260E
:102A3700F6500418E436F650CF750A00750900AE53
:102A470009AF0A74FFC39F74019E402475B7A5752B
:102A5700B7F190024E12001EE0FC90E00012001E3B
:102A6700ECF0780A740126F6500418E436F650CFD5
:102A7700750A00750900AE09AF0A74FFC39F740198
:102A87009E402475B7A575B7F190044E12001EE05D
:102A9700FC90E20012001EECF0780A740126F65052
:102AA7000418E436F650CF750A00750900AE09AF71
:102AB7000A74FFC39F74019E402475B7A575B7F1CB
:102AC70090064E12001EE0FC90E40012001EECF08F
:102AD700780A740126F6500418E436F650CF758F3D
:102AE7000075F51175B62075D940D2AF743A9007C5
:102AF7004EF022900788E0B4AA028003022C37C266
:102B0700AF75D90075B62275F522758F0375B7A510
:102B170075B7F1740090D600F075B7A575B7F17465
:102B27000090D800F075B7A575B7F1740090DA007A
:102B3700F075B7A575B7F1740090DC00F0758F01DB
:102B4700750A00750900AE09AF0A74FFC39F7401C7
:102B57009E402475B7A575B7F190004E12001EE090
:102B6700FC90D60012001EECF0780A740126F6508D
:102B77000418E436F650CF750A00750900AE09AFA0
:102B87000A74FFC39F74019E402475B7A575B7F1FA
:102B970090024E12001EE0FC90D80012001EECF0CE
:102BA700780A740126F6500418E436F650CF750AF1
:102BB70000750900AE09AF0A74FFC39F74019E40F8
:102BC7002475B7A575B7F190044E12001EE0FC906E
:102BD700DA0012001EECF0780A740126F650041889
:102BE700E436F650CF750A00750900AE09AF0A74CE
:102BF700FFC39F74019E402475B7A575B7F1900672
:102C07004E12001EE0FC90DC0012001EECF0780A69
:102C1700740126F6500418E436F650CF758F007508
:102C2700F51175B62075D940D2AF743A90074EF0BA
:102C370022C2AF75D90075F522750A00750900AE75
:102C470009AF0A74FFC39F74019E401F90EE0012E4
:102C5700001EE493FC90004E12001EECF0780A74FC
:102C67000126F6500418E436F650D4750A007509A3
:102C770000AE09AF0A74FFC39F74019E401F90F016
:102C87000012001EE493FC90024E12001EECF07836
:102C97000A740126F6500418E436F650D4750A0073
:102CA700750900AE09AF0A74FFC39F74019E401FE8
:102CB70090F20012001EE493FC90044E12001EECEA
:102CC700F0780A740126F6500418E436F650D475E5
:102CD7000A00750900AE09AF0A74FFC39F74019E0D
:102CE700401F90F40012001EE493FC90064E120061
:102CF7001EECF0780A740126F6500418E436F650F4
:102D0700D475F51175D940D2AF22C2AF75D9007508
:102D1700F522750A00750900AE09AF0A74FFC39F53
:102D270074019E401F90E60012001EE493FC900081
:102D37004E12001EECF0780A740126F6500418E4CF
:102D470036F650D4750A00750900AE09AF0A74FF4C
:102D5700C39F74019E401F90E80012001EE493FC7D
:102D670090024E12001EECF0780A740126F6500409
:102D770018E436F650D4750A00750900AE09AF0A93
:102D870074FFC39F74019E401F90EA0012001EE467
:102D970093FC90044E12001EECF0780A740126F69C
:102DA700500418E436F650D4750A00750900AE09C8
:102DB700AF0A74FFC39F74019E401F90EC0012007E
:102DC7001EE493FC90064E12001EECF0780A740184
:102DD70026F6500418E436F650D475F51175D94027
:102DE700D2AF22C2AF75D90075F522750A007509F1
:102DF70000AE09AF0A74FFC39F74019E401F90DEA7
:102E07000012001EE493FC90004E12001EECF078B6
:102E17000A740126F6500418E436F650D4750A00F1
:102E2700750900AE09AF0A74FFC39F74019E401F66
:102E370090E00012001EE493FC90024E12001EEC7C
:102E4700F0780A740126F6500418E436F650D47563
:102E57000A00750900AE09AF0A74FFC39F74019E8B
:102E6700401F90E20012001EE493FC90044E1200F3
:102E77001EECF0780A740126F6500418E436F65072
:102E8700D4750A00750900AE09AF0A74FFC39F74B1
:102E9700019E401F90E40012001EE493FC90064E32
:102EA70012001EECF0780A740126F6500418E43676
:102EB700F650D475F51175D940D2AF22C2AF75D986
:102EC7000075F522750A00750900AE09AF0A74FF8F
:102ED700C39F74019E401F90D60012001EE493FC0E
:102EE70090004E12001EECF0780A740126F650048A
:102EF70018E436F650D4750A00750900AE09AF0A12
:102F070074FFC39F74019E401F90D80012001EE4F7
:102F170093FC90024E12001EECF0780A740126F61C
:102F2700500418E436F650D4750A00750900AE0946
:102F3700AF0A74FFC39F74019E401F90DA0012000E
:102F47001EE493FC90044E12001EECF0780A740104
:102F570026F6500418E436F650D4750A00750900B1
:102F6700AE09AF0A74FFC39F74019E401F90DC0037
:102F770012001EE493FC90064E12001EECF0780A35
:102F8700740126F6500418E436F650D475F5117519
:102F9700D940D2AF22E51464046006E59964FF6066
:102FA700028031A20F4004D20F8027E51460087415
:102FB700E62514900023F0E513600874F0251390BC
:102FC7000023F0E514B4010280FE751400751300A8
:102FD700C20F8002C20FE5149038FDF828287375D8
:102FE7001400E599B4FF03751301E599B4FE037561
:102FF7001302E599B4FD03751303E599B4FC037552
:103007001304E599B4FA03751305E599B4FB06753E
:103017001401120464E599B4F906751404120464E2
:10302700E599D394E54007E599C394F040028016EB
:103037008599157514027E017F00E515C394E61284
:103047003FE98E0D8F0E900786E4F0A3F0E599D344
:1030570094C44007E599C394E640028028859915F2
:1030670075140374E5C39515F50E750D00AE0DAF18
:103077000E90395A12002EE493F874019390078644
:10308700C8F0A3C8F0D299023511900786E0FEA3D5
:10309700E0FFEFC39400EE94054009EFD394FFEEF1
:1030A70094064013900786E0FEA3E0FF90004E12BF
:1030B700001EE599F0800385996C90078612000E33
:1030C700900786E0FEA3E0FFEFB40106EEB4070227
:1030D700800302331E90074EE0B43C0280030233A4
:1030E7001E75FFA0A20AB35005A20CB3400302321B
:1030F70011C29C90007AE090078CF0900057E09006
:10310700078DF0900062E090078EF0900063E090EA
:10311700078FF0900074E0900790F090007CE090AB
:103127000791F090007DE0900792F0900080E0908A
:103137000793F0900081E0900794F090013AE090B7
:103147000795F090013BE0900796F090013CE090E6
:103157000797F0900090E0900798F0900091E0902A
:103167000799F0900092E090079AF0900093E09012
:10317700079BF0900094E090079CF0900095E090FA
:10318700079DF0900096E090079EF0900097E090E2
:10319700079FF0900099E09007A0F090009AE090C8
:1031A70007A1F090009BE09007A2F090009CE090B0
:1031B70007A3F07400900082F01200AC74AB900784
:0D31C70088F012269574AA900788F0E5584C
:0638FD00022FE6023091EB
:1031D40090391EF82828738012122740800D122877
:0B31E4007E80081229BC8003122AFA2A
:0F391E000231DB0231DD0231E20231E70231EC2E
:1031EF00900788E4F090013AE0700C90013BE0709A
:1031FF000690013CE060028004C20A8002D20A02FB
:10320F003313C29C900078E0900789F090005EE045
:10321F0090078AF090005FE090078BF090007AE0C3
:10322F0090078CF0900057E090078DF0900062E0CF
:10323F0090078EF0900063E090078FF0900074E09D
:10324F00900790F090007CE0900791F090007DE067
:10325F00900792F0900080E0900793F0900081E04B
:10326F00900794F090013AE0900795F090013BE0C1
:10327F00900796F090013CE0900797F0900090E057
:10328F00900798F0900091E0900799F0900092E0ED
:10329F0090079AF0900093E090079BF0900094E0D5
:1032AF0090079CF0900095E090079DF0900096E0BD
:1032BF0090079EF0900097E090079FF0900099E0A4
:1032CF009007A0F090009AE09007A1F090009BE08B
:1032DF009007A2F090009CE09007A3F0740090007C
:1032EF0082F074AB900788F012269574AA90078825
:1032FF00F012274012287E1229BC122AFAD29C758E
:10330F0099FB80FED29C7514007513007599FB0212
:10331F003511900786E0FEA3E0FFEF4E700685990A
:10332F0010750F00900786E0FEA3E0FF74016F4E4B
:10333F00701BAC0FAD10AA0DAB0EED2BFBEC3AFAD8
:10334F008A068B0790004E12001EE599F0900786B3
:10335F0012000E900786E0FEA3E0FF74026F4E701E
:10336F000C1200AC851599751400751300023511F8
:10337F00900786E0FEA3E0FF90004E12001EE59935
:10338F00F090078612000E900786E0FEA3E0FFACD8
:10339F000DAD0E8F028E038C068D079039921200A1
:1033AF002EE493F9740193FEEAD39EEB99400985BD
:1033BF001599751400751300023511900786E0FEFC
:1033CF00A3E0FF90004E12001EE599F090078612C1
:1033DF00000E900786E0FEA3E0FFEFB40006EEB408
:1033EF000102800302351175FFA090001CE0D394F9
:1033FF00C7400B90001CE0C394C8F516801A9000CC
:10340F001CE0D39463400B90001CE0C39464F5164A
:10341F00800690001CE0F516E51675F002A4FFAECD
:10342F00F08F6BEF90004E124001EFFCE0FDEC903F
:10343F000051124001EDFCE0FDEC2DB516028003AA
:10344F000235030FEF90004E124001E56BFFE0FCD9
:10345F00EF900052124001ECFFE0FCEFC39CB51659
:10346F00028003023503E56B900050124001E56BBB
:10347F00FFE0FCEF900053124001ECFFE0FCEF2C5B
:10348F00B51671E56B900054124001E0C39516908C
:10349F00079DF0E56B900055124001E0C395169023
:1034AF00079EF0E56B900058124001E0C39516900F
:1034BF00079FF0E56B900059124001E0C3951690FD
:1034CF0007A0F0E56B90005A124001E0C3951690EB
:1034DF0007A1F0E56B90005B124001E0C3951690D9
:1034EF0007A2F012260B7599F9751864751700125B
:1034FF0025C780FE7599FF7518647517001225C7CB
:02350F0080FE3C
:0939030002332102337F0233CAB2
:1035110022E51390390CF828287302365290078659
:10352100E0FEA3E0FF90001212001EE0F599900763
:103531008612000E900786E0FEA3E0FF74116F4E25
:103541007003751300023652856299023652900754
:1035510086E0FEA3E0FF90004E12001EE0F599EF19
:10356100B40107EEB4070375130090078612000E2D
:07357100023652900787E0CB
:0F390C0002351B02351E02354902354F02357454
:1035780090392DF8282873852499023647852A9989
:10358800023647854499023647854799023647856A
:103598005199023647856099023647855699023611
:1035A80047855899023647756E00900069E07006A5
:1035B800900068E060028016A2A44006E56E44040C
:1035C800F56EA2A54006E56E4402F56E801A9000DD
:1035D8004AE0B40106E56E4410F56E900049E0B487
:1035E8000106E56E4420F56EA207B34006E56E4479
:1035F80001F56EA209B34006E56E4408F56E856EC6
:1036080099803CA210B340077599FAC2108017A29E
:103618000DB3400575990F800B900023E0F5999044
:103628000023E4F0C20D80178542998012854B99DA
:0F363800800D85469980087599FC8003751300F5
:10392D0002357F02358502358B02359102359702BE
:10393D00359D0235A30235A90235AF02360B02368D
:0D394D003002363502363A02363F0236446B
:0B36470090078612000E80031200485E
:03391B0002364F22
:103652002290006BE0B4010385241190006BE0B46A
:103662000203852A1190006BE0B403038544119094
:10367200006BE0B4040385471190006BE0B40503CE
:1036820085511190006BE0B4060385561190006BD2
:10369200E0B4070385581190006CE0FE90006DE0E5
:1036A200C39E500302372990006BE0D39404402C50
:1036B20090006CE0D39511500990006DE0C3951114
:1036C20050028002D20090006CE0D3951150099014
:1036D200006DE0C395115002C200804990006BE07A
:1036E200B4041890006DE0C395115002D20090000E
:1036F2006CE0D395114002C200802A90006CE0C3B6
:103702009511500990006DE0D3951150028002D2BC
:103712000090006CE0D39511500990006DE0C395C4
:10372200115002C200807E90006BE0D39404402CC2
:1037320090006CE0C39511400990006DE0D39511A3
:1037420040028002C20090006CE0C39511400990D3
:10375200006DE0D395114002D200804990006BE0E9
:10376200B4041890006CE0C395115002C20090009E
:103772006DE0D395114002D200802A90006CE0C324
:103782009511400990006DE0D395114002D200904E
:10379200006CE0D39511400990006DE0C395114093
:1037A200028002C2002290006EE0B401038524115F
:1037B20090006EE0B40203852A1190006EE0B4031B
:1037C2000385441190006EE0B40403854711900014
:1037D2006EE0B4050385511190006EE0B4060385D6
:1037E200561190006EE0B4070385581190006FE007
:1037F200FE900070E0C39E500302387E90006EE09F
:10380200D39404402C90006FE0D39511500990009E
:1038120070E0C3951150028002D20290006FE0D393
:1038220095115009900070E0C395115002C20280B8
:103832004990006EE0B40418900070E0C3951150F6
:1038420002D20290006FE0D395114002C202802A98
:1038520090006FE0C395115009900070E0D395116C
:1038620050028002D20290006FE0D395115009906D
:103872000070E0C395115002C202807E90006EE09B
:10388200D39404402C90006FE0C39511400990003E
:1038920070E0D3951140028002C20290006FE0C333
:1038A20095114009900070E0D395114002D2028038
:1038B2004990006EE0B4041890006FE0C395115077
:1038C20002C202900070E0D395114002D202802A17
:1038D20090006FE0C395114009900070E0D39511FC
:1038E2004002D20290006FE0D3951140099000701F
:0B38F200E0C3951140028002C20222D8
:094001002582F58250020583229C
:10002E00EF2F500205832582F582E5833E2EF58360
:01003E00229F
:08000300C3EF9DFFEE9CFE22FD
:08003F000806B60002180622B3
:0D000E00A3E004F07006123FF7E004F022BA
:084013000816B6FF0218162280
:0E3FDB00048007C3CE13CECF13CFD5E0F6225D
:103E8900BC000FBE0008ED8FF084FFADF022E4FE08
:103E9900FF22BE000DEF60FE54F0606F20E70302C1
:103EA9003F3FEAC0E0EBC0E078017A0075F001EE2F
:103EB90020E710EF25E0FFEE33FE0AC5F023C5F039
:103EC90030E7F0EA5407F9096A7A007B00600108D3
:103ED900C3EC9E40167004ED9F4010ED9FFDEC9ED3
:103EE900FCE5F0CA4ACA03F5F08005E5F003F5F0F0
:103EF900C3EE13FEEF13FFD9D77908CACBCAD8D0BE
:103F0900EAFEEBFFD0E0FBD0E0FA22EC8FF084FC74
:103F1900ED54F045F0C48FF084FEEDC454F045F043
:103F2900C48FF084FDEEC4FE54F02DFFEE540F3C17
:103F3900FEADF07C0022790078008FF0EC7E08203D
:103F4900E70DC3CD33CD33C933C9C833C8DEF084D7
:103F590049F9E5F08FF0BE00E6FD7C00E9FFE8FED7
:013F69002235
:0E3FE900F88FF0A4FFE5F0CE88F0A42EFE22A3
:103FBB00600D782B023FC5007830D8FED5E0F82293
:103FCB00EEC0E07E00123E89EFFDEEFCD0E0FE225B
:03000B00023F6A47
:03001B00023F851C
:03002B00023FA0F1
:0300000002400AB1
:09400A0075817375D000020703F3
:0B001E00E5822FF582E5833EF583228A
:0A3FF7000582D5820215831582228F
:103F6A00C0E0C0F0C083C082C0D075D0001206F88D
:103F7A00D0D0D082D083D0F0D0E032C0E0C0F0C040
:103F8A0083C082C0D075D0001206FBD0D0D082D0B8
:103F9A0083D0F0D0E032C0E0C0F0C083C082C0D08D
:103FAA0075D0001206FED0D0D082D083D0F0D0E0F7
:013FBA0032D4
:00000001FF
